S01900006F70656E626C745F73746D3332663734362E73726563F8
S3150800000000000520A54A0008F54A0008F54A000838
S31508000010F54A0008F54A0008F54A000800000000FD
S31508000020000000000000000000000000F54A00087B
S31508000030F54A000800000000F54A0008C109000852
S31508000040F54A0008F54A0008F54A0008F54A000886
S31508000050F54A0008F54A0008F54A0008F54A000876
S31508000060F54A0008F54A0008F54A0008F54A000866
S31508000070F54A0008F54A0008F54A0008F54A000856
S31508000080F54A0008F54A0008F54A0008F54A000846
S31508000090F54A0008F54A0008F54A0008F54A000836
S315080000A0F54A0008F54A0008F54A0008F54A000826
S315080000B0F54A0008F54A0008F54A0008F54A000816
S315080000C0F54A0008F54A0008F54A0008F54A000806
S315080000D0F54A0008F54A0008F54A0008F54A0008F6
S315080000E0F54A0008F54A0008F54A0008F54A0008E6
S315080000F0F54A0008F54A0008F54A0008F54A0008D6
S31508000100F54A0008F54A0008F54A0008F54A0008C5
S31508000110F54A0008F54A0008F54A0008F54A0008B5
S31508000120F54A0008F54A0008F54A0008F54A0008A5
S31508000130F54A0008F54A0008F54A0008F54A000895
S31508000140F54A0008F54A0008F54A0008F54A000885
S31508000150F54A0008F54A0008F54A0008F54A000875
S31508000160F54A0008F54A0008F54A0008F54A000865
S31508000170F54A0008F54A0008F54A0008000000009C
S31508000180F54A0008F54A0008F54A0008F54A000845
S31508000190F54A0008F54A0008F54A0008F54A000835
S315080001A0F54A0008F54A0008F54A0008F54A000825
S315080001B0F54A0008F54A0008F54A0008F54A000815
S30D080001C0F54A0008F54A00089B
S315080001C810B5054C237833B9044B13B10448AFF37B
S315080001D800800123237010BDC00000200000000025
S315080001E8C44F000808B5034B1BB103490348AFF3CE
S315080001F8008008BD00000000C4000020C44F0008A5
S3150800020872B6704762B670472DE9F04184B0044665
S315080002180D4617469846684602F022FE164B02997E
S31508000228A3FB01318909002201E00132D2B2112A61
S315080002381DD8124B13F8120003EB420393F801E09A
S3150800024800EB0E0303FB0443B1FBF3FC03FB1C168C
S31508000258002EEAD11FFA8CF32B80013B9BB2B3F52B
S31508000268806FE2D2387088F800E0012000E00020AC
S3150800027804B0BDE8F08100BFD34D621004500008F1
S3150800028870B58CB00022ADF82E208DF82D200CAB59
S3150800029803F8042D0DF12D020DF12E014FF4FA7015
S315080002A8FFF7B2FF002835D01D4C1E4B23600025EA
S315080002B825766576A5760126E67625776577A56097
S315080002C8E5609DF82D30013B1B0423619DF82C3011
S315080002D8013B1B056361BDF82E306360204601F0BB
S315080002E808F90695079508964CF6E0430193029592
S315080002F84FF6E073039304230493059509960E2392
S315080003080A9301A9204601F09BF9204601F02EFA26
S315080003180CB070BDB521044800F034FDC4E700BF31
S31508000328DC00002000640040DC4F000810B588B0E7
S3150800033840F2E1730293002304930593069101ABF7
S31508000348024602A90B4801F03FFA08B108B010BDE9
S3150800035800F026FB00F132040199064801F0A9FAD3
S315080003680028F3D000F018FE00F01AFB8442F3D2F6
S31508000378ECE700BFDC00002010B588B00C46034641
S3150800038801AA00210A4801F0A6FA50B940F26763A3
S31508000398019A9A4201D0002004E0039B13B9012070
S315080003A800E0002008B908B010BD059B2370FAE7DD
S315080003B8DC00002008B5FFF723FF08BD10B500F0DC
S315080003C8FBF900B910BD00F0E7FF0028FAD000F0E5
S315080003D88DFD00F0BDFA01F02FF800F0F1F9054B94
S315080003E80340054A936000F0EBF94468FFF70AFFF3
S315080003F8A047E7E780FFFF1F00ED00E070B508E0BB
S31508000408461C4D1C0B78037000F0C6FD304629467D
S315080004182246531E9CB2002AF2D170BD38B505464D
S31508000428002401E00134E4B2062C15D800F0B4FD26
S3150800043804EB44029300094AD358AB42F2D804EBBA
S3150800044844029100054A0A44526813449D42E9D277
S31508000458024B0B44187A38BDFF2038BD28500008CF
S3150800046808B5C1F3080353B90368994209D040F897
S31508000478041B4FF40072FFF7C1FF012008BD0020D6
S3150800048808BD012008BD2DE9F041074601F0A2FB89
S3150800049800247F2C14D83E68A30006EB03083B44C7
S315080004A85D6800F079FD2A4600234146022001F0DE
S315080004B8E7FB38B956F824309D4209D10134E8E7F4
S315080004C8012400E0002401F09DFB2046BDE8F081E8
S315080004D80024F8E738B50D460B4B984208D0044671
S315080004E80A4B994206D0FFF7CEFF20B9002407E049
S315080004F8074C00E0044C29462046FFF7B1FF08B12F
S31508000508204638BD0024FBE70803002000800008C1
S31508000518040100202DE9F04106460C4617461D46FB
S31508000528DFF8748001EA08080368B3F1FF3F0DD0C5
S315080005383368984505D041463046FFF7CBFF06464F
S3150800054828B33368E41A344404340CE04146FFF708
S3150800055887FF03460028EBD116E017F8013B04F895
S31508000568013B013D0FD000F017FD331DE31AB3F523
S31508000578007FF2D308F500713046FFF7ABFF064651
S3150800058838B1041DE9E701231846BDE8F0810023C0
S31508000598FAE70023F8E700BF00FEFFFF70B586B04C
S315080005A804460D4600230193884205D801262CB136
S315080005B8072D04D9002602E00026F8E7002616B912
S315080005C8304606B070BD0023029302230593012323
S315080005D8049301F0FFFAAC420BD800F0DDFC039453
S315080005E801A902A801F0CEFB10B90134E4B2F2E77A
S315080005F8002601F007FBE3E74FF0FF33024A1360D2
S31508000608024A1360704700BF04010020080300204F
S3150800061870B54B1E144C241AA34201D9002070BD8C
S3150800062816460D460446FFF7F9FEFF2818D028197E
S315080006380138FFF7F3FEFF2814D00C4B23400C4A69
S31508000648934206D02B46324621460A48FFF762FFF0
S3150800065870BD2B46324621460748FFF75BFF70BD3B
S31508000668002070BD002070BDFFFF0F0800FEFFFFC9
S315080006780080000804010020080300204A1E0D4BCC
S315080006881B1A9A4201D90020704770B50C460546D0
S31508000698FFF7C4FE064660190138FFF7BFFEFF28B4
S315080006A818BFFF2E01D1002070BD01463046FFF75E
S315080006B875FF70BDFFFF0F08104B1B68B3F1FF3FAE
S315080006C81AD000B583B00D4A536891680B44D168AF
S315080006D80B4411690B4451690B4491690B44D2695F
S315080006E813445B4202AA42F8043D04210448FFF772
S315080006F88FFF03B05DF804FB01207047080300204C
S31508000708C88100080D4B1B680D4A126813440D4A28
S31508000718126813440C4A126813440C4A12681344A4
S315080007280B4A126813440B4A126813440A4A126899
S31508000738D34201D000207047012070470080000886
S3150800074804800008088000080C800008108000084B
S315080007581480000818800008C881000808B50C4BE2
S315080007681B68B3F1FF3F04D00948FFF78CFE034620
S3150800077850B1084B1B68B3F1FF3F07D00548FFF790
S3150800078882FE034600B10123184608BD0123FBE78C
S31508000798080300200401002000487047008000086C
S315080007A808B5FFF729FF08BD08B5FFF731FF08BDEB
S315080007B808B5FFF763FF08BD08B5FFF7A3FF08BD2F
S315080007C808B5FFF7E9FF08BD08B5FFF775FF034643
S315080007D808B9184608BDFFF7C1FF0346F9E7000040
S315080007E8074BDB6913F0200F06D0012333B1044BFE
S315080007F85B6A0370012070470023F7E700207047FB
S315080008080048004010B50B4B986200F0C9F800F193
S315080008180A0407E0012363B900F0BEFB00F0C0F83C
S31508000828844206D3034BDB6913F0800FF2D1002309
S31508000838F1E710BD0048004010B588B04FF4614391
S31508000848019300230293039304930C2205920693BB
S315080008580793054C01A9204602F0AAFC236843F031
S315080008680103236008B010BD0048004070B506466D
S315080008780D46402904D82846FFF7C4FF00240BE094
S315080008888121074800F07EFAF5E700F085FB305D20
S31508000898FFF7B8FF0134A4B2ABB29C42F5D370BDDA
S315080008A87C50000870B5254B1C78BCB92448FFF75E
S315080008B897FF012801D0204670BD214B1B78013BC4
S315080008C8DBB23F2BF7D800F06BF81E4B18600022F6
S315080008D81D4B1A700122194B1A70ECE706460D468D
S315080008E8194B1B78013316481844FFF779FF044655
S315080008F801280AD000F054F8124B1B686433984252
S3150800090819D900240D4B1C70D5E70F4B1A780132FC
S31508000918D2B21A700A4B1B789A4201D00024CAE749
S315080009280A493046FFF76AFD0022044B1A70064B3F
S315080009381B782B70BFE70024BDE700BF4D050020D4
S315080009480C050020500500204E0500200D05002046
S315080009580022014B1A60704710E000E008B5FFF75F
S31508000968F7FF054B054A5A6000229A600521196067
S31508000978034B1A6008BD00BF10E000E0BF4B030038
S3150800098854050020044B1B6813F4803F03D0034A20
S31508000998136801331360704710E000E0540500201F
S315080009A808B5FFF7EFFF014B186808BD5405002086
S315080009B808B5FFF7F5FF08BD70470000094B03F1B6
S315080009C81801002232B19A7400225A61054A064B68
S315080009D81A6070479A745961183318310132D2B2BD
S315080009E8F0E700BF98050020C80500200A4B1B68D9
S315080009F883B110B45C69084A146019749860D860A1
S31508000A0800225A741860013908445860987C5DF8C1
S31508000A18044B7047FF207047C805002038B50446C0
S31508000A280D46012804D94FF4E071124800F0AAF9D6
S31508000A3862002244D100104B0B445A7C1B7C9A4214
S31508000A4813D00D4B0B44DA6815705A7C01325A7468
S31508000A58DA680132DA605B689A4208D9064A0846B3
S31508000A6851580244D160012038BD002038BD012004
S31508000A7838BD00BFA85000089805002008B50146EB
S31508000A88024B1878FFF7CAFF08BD00BFCC0500203F
S31508000A9838B504460D46012804D94FF4F1711348B0
S31508000AA800F070F904EB4403DA00114B13445B7C3D
S31508000AB8BBB162002244D1000D4B0B449A681278E8
S31508000AC82A705A7C013A5A749A6801329A605B68A5
S31508000AD89A4208D9064A08465158024491600120A4
S31508000AE838BD002038BD012038BD00BFA850000811
S31508000AF89805002008B50146024B1878FFF7C8FF85
S31508000B0808BD00BF1006002010B50446012804D900
S31508000B1840F20221044800F035F904EB4404E200E7
S31508000B28024B1344587C10BDA850000898050020AD
S31508000B3838B5FFF743FF1A4C4021601CFFF756FFEC
S31508000B482070184D4021681CFFF750FF287023783D
S31508000B58FF2B1BD0FF2819D0134C00221349204617
S31508000B6803F02AF91249204603F04FF9012000F04C
S31508000B782AFC204603F050F9D4F8980201F0ADFD96
S31508000B8800F02CF9B0F5FA6F05D338BD8521094868
S31508000B9800F0F8F8E0E74FF4FA6000F019F9F4E71E
S31508000BA8CC050020100600205406002070000020FE
S31508000BB80C000020A850000810B5064CD4F8980276
S31508000BC801F09DFD204603F00EF9002000F0FBFB1E
S31508000BD810BD00BF5406002070B506460D463F29CD
S31508000BE80AD82846FFF74AFF012803D0BD210E4830
S31508000BF800F0C8F8002406E0B9210B4800F0C2F84E
S31508000C08EFE70134A4B2ABB29C420BD200F0C4F9A8
S31508000C18305DFFF733FF0128F3D0C621024800F0FC
S31508000C28B1F8EEE770BD00BFA850000870B50646D3
S31508000C380D461F4BD3F8980201F0E2FA1D4B1C78B3
S31508000C489CB91D48FFF756FF012801D0204670BDFC
S31508000C58194B1B78013BDBB23E2BF7D80122154B03
S31508000C681A700022154B1A70F0E7144B1B780133DB
S31508000C7811481844FFF73EFF0446012801D000240E
S31508000C88E4E70E4B1A780132D2B21A700A4B1B786F
S31508000C989A4201D00024D9E709493046FFF7AEFB46
S31508000CA80022044B1A70054B1B782B70CEE700BF41
S31508000CB85406002030090020F008002031090020D9
S31508000CC8F108002030B583B0144B1878FFF71CFFDD
S31508000CD808B30546402800D94025002405E09DF8B4
S31508000CE807200F4B1A550134E4B2A5420DD90DF168
S31508000CF807010A4B1878FFF7CBFE0128EFD04FF407
S31508000D08A371084800F03EF8E9E7ABB2044A812126
S31508000D18054804F08EF803B030BD00BFCC050020A6
S31508000D2858050020A85000085406002070B5044647
S31508000D3803F054FF064621460F4804F028F885B202
S31508000D48002401E00134A4B2AC420CD2315D0B4B4D
S31508000D581878FFF763FE0128F4D04FF4B4710848F1
S31508000D6800F010F8EEE703F039FF402302460121A8
S31508000D78014804F066F870BD5406002010060020E5
S31508000D88A850000808B500F007F9FCE708B500F010
S31508000D98F7F8012803D00B4B1B78012B00D008BDA8
S31508000DA8FFF7FEFD084B1B68084A1268134403F54B
S31508000DB8FA739842F3D30022024B1A70FFF7FEFA29
S31508000DC8EDE700BF38090020340900203C09002057
S31508000DD8014B1860704700BF34090020014B18689A
S31508000DE8704700BF3409002008B5054B1B78012B4E
S31508000DF800D008BDFFF7D4FD024B1860F9E700BF1D
S31508000E08380900203C09002008B50122034B1A704E
S31508000E18FFF7EAFFFFF7BAFF08BD00BF3809002049
S31508000E2808B5FFF7C7FA00F0B3F8FFF797FDFFF71D
S31508000E38B7FC00F00DF8FFF7E7FF08BD08B500F0A6
S31508000E48ABF8FFF79FFD00F017F8FFF79FFF08BDFF
S31508000E5810B500F00FFAFFF713FA064C01232370B2
S31508000E68FFF7EAFC00232370FFF762FE02232370CC
S31508000E7810BD00BF0000002000B583B00DF10701C2
S31508000E881848FFF779FA012810D00DF10701154817
S31508000E98FFF708FD012812D00DF107011148FFF7E1
S31508000EA8C5FE012814D003B05DF804FB01220E4BD9
S31508000EB81A709DF807100B4800F0FCF9E5E70022C0
S31508000EC8094B1A709DF80710064800F0F3F9E3E78E
S31508000ED80222054B1A709DF80710024800F0EAF935
S31508000EE8E1E700BF400900200000002008B5FFF729
S31508000EF863FE08BD38B504460D460E4B1B78012B14
S31508000F0809D00C4B1B7853B10A4B1B78022B0BD014
S31508000F1800F0C8F938BDC9B2FFF708FAF1E7E9B22F
S31508000F282046FFF7A3FCEFE7E9B22046FFF754FE91
S31508000F38EEE700BF00000020074B1B78022B05D000
S31508000F48032B05D0012B05D0402070473F2070475A
S31508000F58002070470820704700000020074B1B78C0
S31508000F68022B05D0032B05D0012B05D0402070474E
S31508000F783F2070470020704708207047000000206F
S31508000F8808B500F085F9034600B10123184608BDDF
S31508000F9808B500F00FFA08BD08B500F010FA08BD44
S31508000FA80022014B5A70704780090020034BFE2225
S31508000FB8DA7018710222A3F84420704780090020C5
S31508000FC810B5054C00232370FFF7EAFFFF23E370EB
S31508000FD80123A4F8443010BD80090020064BFF22DF
S31508000FE8DA7000221A71597859719A71DA711A7277
S31508000FF80622A3F8442070478009002008B5002077
S31508001008FFF7D4FF08BD0000074BFF22DA70074A2E
S315080010189A6400221A715A719A710722C3F807202E
S315080010280822A3F84420704780090020D0500008F9
S31508001038044BFF22DA7042689A640122A3F8442016
S31508001048704700BF8009002008B53120FFF7AEFFBA
S3150800105808BD000038B5084CFF23E3700025257144
S315080010686571FFF769FFA071E57125726572072337
S31508001078A4F8443038BD00BF8009002038B5FFF70A
S315080010888FFF0E4C01252570FF23E370102323716B
S3150800109800236371FFF750FFA071FFF75FFFE07148
S315080010A8FFF75CFFC0F3072020726572A572082354
S315080010B8A4F84430FFF774FB38BD00BF8009002048
S315080010C838B505464478FFF737FF0138844210DCFF
S315080010D80A4C6A78A16C201DFFF790F9FF23E37084
S315080010E86A78A36C1344A3646B780133A4F8443074
S315080010F838BD2220FFF75AFF38BD00BF80090020F7
S3150800110838B504464578FFF717FF0138854211DCDC
S3150800111861680A4DA9646278281DFFF76FF9FF23ED
S31508001128EB706278AB6C1344AB6463780133A5F84B
S31508001138443038BD2220FFF739FF38BD8009002022
S31508001148F8B505461746002406E015F8013B1C4481
S31508001158E4B2FFF721FF31464E1E0029F5D13C605F
S315080011680120F8BD10B5084CFF23E370E21D41685D
S31508001178A06CFFF7E5FF207100236371A3710823AC
S31508001188A4F8443010BD00BF8009002038B50546CC
S315080011980D4B9C6CFFF7D0FE6A1C411E2046FFF7D4
S315080011A803FB60B1084CFF23E370FFF7C5FE01385F
S315080011B8A36C0344A3640123A4F8443038BD312042
S315080011C8FFF7F4FE38BD00BF8009002038B504468D
S315080011D84578FFF7B1FE023885420EDC114BFF222F
S315080011E8DA700122A3F84420617851B9FFF7ECFABE
S315080011F890B93120FFF7DAFE38BD2220FFF7D6FE70
S3150800120838BDA21C074B986CFFF7CEFA28B161784F
S31508001218044A936C0B44936438BD3120FFF7C6FE25
S3150800122838BD00BF8009002008B54168074B986C8F
S31508001238FFF7BEFA30B1054BFF22DA700122A3F890
S31508001248442008BD3120FFF7B1FE08BD80090020FB
S3150800125808B5FFF7B3F8034BFF22DA700122A3F8A3
S31508001268442008BD8009002008B589B2FFF742FE68
S3150800127808BD0000054B00221A709A6483F84320BB
S31508001288A3F844209A705A70704700BF8009002056
S31508001298034B1B780BB1012070470020704700BF2D
S315080012A8800900200022024B83F84320704700BFBC
S315080012B88009002008B50378FF2B04D0354A127830
S315080012C8012A14D008BDFFF7D9FE324B93F84330EC
S315080012D8012B5AD02F4BB3F944100029F2DD1846D2
S315080012E8012380F843300330FFF7BEFFEAE7C93B1E
S315080012F8352B46D8DFE803F03345454245453F36A2
S315080013083C3945454545454545454545454545458C
S315080013184545454545454545454545454545454567
S315080013284545241E1B2145454527452A2D30FFF7E7
S31508001338C7FECAE7FFF7E4FEC7E7FFF779FEC4E783
S31508001348FFF710FFC1E7FFF75FFEBEE7FFF756FE98
S31508001358BBE7FFF743FEB8E7FFF732FEB5E7FFF747
S3150800136815FFB2E7FFF732FFAFE7FFF773FEACE703
S31508001378FFF75AFFA9E7FFF76BFFA6E7FFF764FE33
S31508001388A3E72020FFF712FE9FE71020FFF70EFEBF
S31508001398A0E700BF8009002008B5054B1B6913F4B0
S315080013A8005F01D0002008BD00F03EF8012008BD06
S315080013B80008024008B5642000F008F808BD08B51A
S315080013C800F00AF808BD704770477047014B188047
S315080013D8704700BFCC09002008B5FFF7E1FA0E4BA5
S315080013E81B6898420FD30D4B1B786BB901220B4B20
S315080013F81A7080220A4B9A61FFF7D2FA094B1B88A2
S315080014081844054B186008BD0022044B1A704FF49F
S315080014180002034B9A61EFE7D0090020CE090020A5
S3150800142800040240CC0900204FF40002014B9A61DF
S31508001438704700BF0004024010B5094B4FF0FF3251
S315080014481A6200241C625A625C621A611C615A613B
S315080014585C619A619C6103F0DDFA204610BD00BF05
S315080014680038024010B504460E4B18784FF47A73C4
S31508001478B3FBF0F30C4A1068B0FBF3F000F008FB76
S3150800148868B90F2C01D9012010BD002221464FF05A
S31508001498FF3000F0CDFA054B1C60002010BD012076
S315080014A810BD00BF0100002008000020040000202D
S315080014B808B5032000F0AAFA0020FFF7D3FF03F0C7
S315080014C803FA002008BD000038B50446FFF770FA8D
S315080014D80546B4F1FF3F02D0044B1B781C44FFF7BE
S315080014E867FA401B8442FAD838BD00BF01000020BD
S315080014F87047002800F0A18038B5044690F82030D7
S31508001508D3B12268136823F002031360FFF750FA71
S31508001518054623685A6812F0020F10D0FFF748FAF2
S31508001528401B0A28F5D9636A43F400336362052326
S3150800153884F82030012038BDFFF7DAFFE1E71A689A
S3150800154842F001021A60FFF733FA054623685A681B
S3150800155812F0010F0DD1FFF72BFA401B0A28F5D90F
S31508001568636A43F400336362052384F82030012054
S3150800157838BD227E012A3DD01A6822F080021A60F8
S31508001588637E012B3BD02268136823F0400313605F
S31508001598A37E012B39D02268136823F02003136031
S315080015A8E37E012B37D02268136843F010031360D3
S315080015B8237F012B35D02268136823F008031360AC
S315080015C8637F012B33D02268136823F00403136062
S315080015D82168A368E26813432269134362691343BF
S315080015E86268013A1343CB6100206062012384F8DC
S315080015F8203038BD1A6842F080021A60C0E72268AF
S31508001608136843F040031360C2E72268136843F07F
S3150800161820031360C4E72268136823F010031360D5
S31508001628C6E72268136843F008031360C8E7226808
S31508001638136843F004031360CAE7012070470000E3
S3150800164890F82030013BDBB2012B05D9436A43F4F5
S31508001658802343620120704770B4434BD3F80022B5
S3150800166842F00102C3F80022D3F8002222F47C5281
S31508001678C3F80022D3F80022486A42EA0022C3F8CF
S3150800168800224A6902F01F02012000FA02F2D3F882
S315080016981C42D0430440C3F81C42CB69B3B9324B49
S315080016A8D3F80C420440C3F80C424C69CE688D88BE
S315080016B845EA0645483443F834504D698E680C881F
S315080016C844EA0644483503EBC5035C60CB69012B3D
S315080016D81DD08B69002B32D1234CD4F80432034031
S315080016E8C4F804320B698BBB1F4BD3F8144220404D
S315080016F8C3F814020B6A012B2FD01B4AD2F8003202
S3150800170823F00103C2F80032002070BC7047164B5C
S31508001718D3F80C421443C3F80C424C690E688D88FA
S3150800172845EA0645483443F834504D698E688C892D
S3150800173844EA0644483503EBC5035C60C9E70A4C26
S31508001748D4F804321343C4F80432CBE70648D0F871
S3150800175814321343C0F81432CCE7034BD3F81C12DF
S315080017680A43C3F81C22C8E70064004038B590F855
S315080017782030DBB2012B05D0436A43F400234362C9
S31508001788012038BD0446022380F820300268136811
S3150800179823F001031360FFF70BF9054623685B6816
S315080017A813F0010F0DD0FFF703F9401B0A28F5D9E6
S315080017B8636A43F400336362052384F82030012002
S315080017C838BD0020606238BD70B490F820400568BE
S315080017D8AD68013CE4B2012C06D9436A43F4802378
S315080017E84362012070BC704715F0E05F5BD0C5F313
S315080017F80165022D3ED80124AC401C608B68002B7D
S315080018083ED104680E68CB6843EA465605F11803C4
S315080018181B01E65003680C6905F1180603EB061365
S315080018285C600B7D012B36D00468D17993791B044B
S3150800183843EA0163517943EA012311790B432E01DF
S315080018483444C4F88C310168D47893781B0443EA85
S315080018580463547843EA0423127813433144C1F8DD
S315080018688831026818352D01535943F0010353513D
S315080018780020B7E7436A43F4000343620120B1E74F
S3150800188804684E6843EAC603CE68334305F118066A
S315080018983601A351BEE7036803EB0613596841F4FA
S315080018A880715960C0E7436A43F400134362012014
S315080018B898E790F82030013BDBB2012B01D90020CC
S315080018C8704703689B68890631EA030301D001203B
S315080018D870470020704730B490F82040013CE4B2C5
S315080018E8012C06D9436A43F480234362012030BC9D
S315080018F8704700296FD10468E46814F0030F64D0B0
S31508001908056801F11B0424012C5904F004049460A9
S31508001918002C6BD1056801F11B0424012C59640DB0
S315080019281460056801F11B0424012D59C5F3400507
S31508001938D560056825446D6805F00F0515610568C5
S3150800194825446D68C5F30725956105682C446468C0
S31508001958240C546104680A011444D4F8B8411C706C
S3150800196804681444D4F8B841C4F307245C700468BE
S315080019781444D4F8B841C4F307449C700468144462
S31508001988D4F8B841240EDC7004681444D4F8BC4171
S315080019981C7104681444D4F8BC41C4F307245C7168
S315080019A804681444D4F8BC41C4F307449C71046819
S315080019B82244D2F8BC21120EDA71F9B90268D36842
S315080019C843F02003D360002091E7436A43F40013E9
S315080019D8436201208BE70468246914F0030F8FD14A
S315080019E8436A43F400134362012080E7056801F15E
S315080019F81B0424012C59E408546092E70268136909
S31508001A0843F020031361002071E700000649CB68FC
S31508001A1823F4E0631B041B0C000200F4E060034394
S31508001A28024A1A43CA60704700ED00E00000FA054A
S31508001A3830B4144BDB68C3F30223C3F10704042C40
S31508001A4828BF04241D1D062D13D9033B012505FAB5
S31508001A5804F4013C2140994005FA03F3013B13407D
S31508001A681943002807DB0901C9B2074B195430BCCA
S31508001A7870470023EAE700F00F000901C9B2034BD3
S31508001A881954F4E700ED00E000E400E014ED00E086
S31508001A980138B0F1807F0AD2064B5860F021064A11
S31508001AA882F823100020986007221A6070470120E0
S31508001AB8704700BF10E000E000ED00E010B40A49E6
S31508001AC80C6924F440740C610C6944F440740C6184
S31508001AD80C6944F001040C6102604360BFF34F8F40
S31508001AE85DF8044B704700BF003C0240084B1A6972
S31508001AF822F440721A611A6942F400721A611A6964
S31508001B0842F001021A610160BFF34F8F704700BFA8
S31508001B18003C0240084B1A6922F440721A611A6995
S31508001B2842F480721A611A6942F001021A61018048
S31508001B38BFF34F8F704700BF003C0240074B1A6936
S31508001B4822F440721A611A691A611A6942F0010286
S31508001B581A610170BFF34F8F704700BF003C0240FF
S31508001B681A4BDB6813F0020F04D0194A936943F03D
S31508001B7820039361154BDB6813F0100F04D0144A41
S31508001B88936943F010039361104BDB6813F0200F39
S31508001B9804D00F4A936943F0080393610B4BDB683B
S31508001BA813F0400F04D00A4A936943F0040393617B
S31508001BB8064BDB6813F0800F04D0054A936943F097
S31508001BC802039361F222014BDA607047003C024037
S31508001BD8DC090020094B1B69002B01DB0020704734
S31508001BE8064B074A5A6002F188325A601B69002B6D
S31508001BF801DB002070470120704700BF003C024007
S31508001C0823016745034A136943F00043136100201B
S31508001C18704700BF003C024038B504460022164B00
S31508001C289A61FEF7C5FE0546144BDB6813F4803F38
S31508001C380AD0B4F1FF3FF7D0CCB1FEF7B9FE401B86
S31508001C488442F1D2032038BD0C4BDB6813F0F20F3F
S31508001C5809D10A4BDB6813F0010F0AD00122074B9A
S31508001C68DA60002038BDFFF77BFF012038BD032066
S31508001C7838BD002038BD00BFDC090020003C024002
S31508001C882DE9F0411E4C247D012C03D1022420465F
S31508001C98BDE8F081984617460E4605460122184BB8
S31508001CA81A754CF25030FFF7B7FF044698B9032D5A
S31508001CB807D8DFE805F00214191EF9B23046FFF70F
S31508001CC83DFF4CF25030FFF7A7FF04460D4A13694B
S31508001CD823F0010313610022094B1A75D7E7B9B235
S31508001CE83046FFF717FFECE739463046FFF7FEFEA2
S31508001CF8E7E73A4643463046FFF7E0FEE1E700BF26
S31508001D08DC090020003C0240084B1A6922F440729C
S31508001D181A611A6942F004021A611A6942EA00202D
S31508001D2840F480301861BFF34F8F7047003C02407B
S31508001D3809B3012921D002291AD04FF44071104B52
S31508001D481A6922F440721A611A690A431A611A69E9
S31508001D5822F0F8021A611A6942EAC00040F0020045
S31508001D6818611A6942F480321A61BFF34F8F7047B7
S31508001D784FF40071E3E70021E1E74FF48071DEE7ED
S31508001D88003C0240214B1B7D012B02D10222104642
S31508001D98704770B50E46044601221C4B1A754CF25C
S31508001DA85030FFF739FF024658BB4FF0FF33336010
S31508001DB82368012B16D06568A36861680B449D42A1
S31508001DC81FD2217B2846FFF7B3FF4CF25030FFF7A6
S31508001DD823FF0F4A136923F07A031361024678B979
S31508001DE80135E9E7207BFFF78FFF4CF25030FFF704
S31508001DF813FF024606490B6923F004030B6100E04A
S31508001E0835600021014B1975104670BDDC090020A4
S31508001E18003C02402DE9F04782B0D0F80080CA009D
S31508001E28521A930003445A6D1B6D9A4255D8C146F7
S31508001E389B1AC1EBC104A2000244526C934200D813
S31508001E481A460C46074602F1030A4FEA9A0A15E0AB
S31508001E5806F1030A4FEA9A0AE3001B1B9D003D4454
S31508001E68A96C3B7C0093B3B2E2B2404601F05AFD36
S31508001E78AB6C3344AB646B6D1E446E6509EB441357
S31508001E8803F510639B699BB29A4512D8E3001B1B9E
S31508001E989A003A44516D136D99420AD24BB15B1AAE
S31508001EA8C4EBC4018A003A44566CB342D0D81E46DD
S31508001EB8CEE7E3001B1B980007443A6D7B6D9A42F0
S31508001EC80FD804F00F040123A340D8F8344824EAAD
S31508001ED80304C8F83448002000E0012002B0BDE831
S31508001EE8F0870020FAE77047F0B58BB0002800F0B5
S31508001EF88A80044690F8BD33F3B1032384F8BD33CA
S31508001F08206801F0C5FA254655F8107B6E460FCDB0
S31508001F180FC60FCD0FC695E8030086E80300231DF4
S31508001F280ECB384601F0FAF958B1022384F8BD33C6
S31508001F38012528460BB0F0BD80F8BC33FFF7D3FF60
S31508001F48DBE70021206801F0A9FA002315E0D9008B
S31508001F58C81A82002244012082F83D0082F83C30E3
S31508001F68A2F84230002082F83F0050649064CA1AEA
S31508001F789100214408650133DBB26568AB42E6D3B4
S31508001F88002315E0D800C11A8A002244002182F8E5
S31508001F98FD1182F8FC3182F8FF11C2F80412C2F862
S31508001FA80812C21A90002044C0F810120133DBB296
S31508001FB89D42E7D8254655F8107B6E460FCD0FC6C5
S31508001FC80FCD0FC695E8030086E80300231D0ECB40
S31508001FD8384601F0A9FA054660B9002384F838306E
S31508001FE8012384F8BD33636A012B08D0206801F001
S31508001FF850FE9EE7022384F8BD33012599E720465B
S3150800200800F01CFDF2E7012593E7704790F8BC330A
S31508002018012B01D10220704710B50446012380F828
S31508002028BC33006801F029FE206801F02BFA00206D
S3150800203884F8BC0310BD38B590F8BC33012B02D11F
S315080020480225284638BD0446012380F8BC330068B3
S3150800205801F01EFA206801F0DCFD054620B10023D0
S3150800206884F8BC330125ECE7206801F012FE00234A
S3150800207884F8BC33E5E768B110B50446032380F84D
S31508002088BD33FFF7D8FF2046FFF7BFFF002084F8C7
S31508002098BD0310BD0120704770B505460E46036896
S315080020A8196C03EB461303F53064A3680269012A21
S315080020B807D0364A914257D0F1B202F09BFD00206C
S315080020C870BD13F0080F14D0314A914205D913F49C
S315080020D8004F02D04FF40043A360284602F082FD61
S315080020E805F571720121286801F030FE0823A360FE
S315080020F8E5E713F0200F30D113F0280FDFD1244A73
S31508002108914202D913F4004F2AD1F200921B930088
S315080021182B44D3F804222169C1F31201521AC3F8D1
S315080021281422D3F80412D3F808220A44C3F808225A
S31508002138F1B2284602F05EFD002EC0D1C6EBC606EF
S31508002148B3002B44D3F81032002BB8D105F57172B9
S315080021580121286801F0FAFDB1E72023A360AEE75C
S315080021684FF40043A360AAE713F4004F09D113F00C
S31508002178200F01D02023A360F1B2284602F03AFDC9
S315080021889DE74FF40043A36099E700BF0A31544F0F
S315080021980A30544F38B5044603681D6C03EB4111E1
S315080021A801F530618A680369012B0DD0124B9D42EF
S315080021B814D0204602F016FD104B9D4202D9236919
S315080021C8012B12D0002038BD0C4B9D42F1D912F4D0
S315080021D8004FEED04FF400438B60EAE712F4004F45
S315080021E8E7D04FF400438B60E3E704F571720121E9
S315080021F8206801F0ABFDE5E70A31544F0A30544F21
S315080022082DE9F84F04460568284601F07EFD08B111
S31508002218BDE8F88FA8460746206801F046FD00285D
S31508002228F6D0206801F041FD10F0020F04D02268AC
S31508002238536903F002035361206801F036FD10F470
S31508002248002F40F092803E46206801F02EFD10F4DB
S31508002258802F40F0DC80206801F027FD0028C0F2B6
S315080022684A81206801F021FD10F4006F0AD0D5F8DC
S31508002278083813F0010F40F058812268536903F4AF
S3150800228800635361206801F010FD10F0006F15D047
S315080022982268536903F00063536194F8F433002BFA
S315080022A840F04781012184F8F41323685B6DC3F372
S315080022B88303C4F8F833204600F0D4FB206801F0FD
S315080022C8F4FC10F4805F40F03881206801F0EDFCDA
S315080022D810F4005F40F08A81206801F0E6FC10F0EF
S315080022E8100F14D02268936923F0100393612F6A9C
S315080022F807F00F08C7F34343022B00F08F81062B1C
S3150800230800F0AD812268936943F010039361206851
S3150800231801F0CBFC10F0080F40F0B581206801F0F9
S31508002328C4FC10F4801F40F0B781206801F0BDFC9A
S3150800233810F4001F40F0BA81206801F0B6FC10F0CE
S31508002348804F40F0BD81206801F0AFFC10F0040F03
S315080023583FF45EAF23685D6815F0040F40F0B98155
S3150800236823685A6815435D6052E7206801F0A1FCA6
S3150800237881463E4624E008EB46130122C3F8082B9B
S3150800238831462046FFF788FE29E031462046FFF702
S3150800239801FF08EB46130822C3F8082B22E008EBCE
S315080023A846132022C3F8082B1AF4005F05D008EB59
S315080023B846134FF40052C3F8082B01364FEA590959
S315080023C8B9F1000F3FF440AF19F0010FF5D0F1B29B
S315080023D8206801F07EFC824610F0010FCBD11AF076
S315080023E8080FD2D11AF0100F04D008EB46131022A2
S315080023F8C3F8082B1AF0200FD6D02369012BCED1A3
S3150800240804F571720121206801F0A0FCC7E720686D
S3150800241801F057FC81463E462EE0F200921B9300D7
S315080024282344596C9A6C0A449A6448E01AF0080FCF
S3150800243804D008EB46130822C3F808291AF0100F27
S3150800244804D008EB46131022C3F808291AF0400FDF
S3150800245804D008EB46134022C3F808291AF0020FDD
S3150800246804D008EB46130222C3F808291AF0800F8D
S315080024783CD101364FEA5909B9F1000F3FF4EBAEE2
S3150800248819F0010FF5D05FFA86FB5946206801F066
S3150800249829FC824610F0010FC8D006F00F03012167
S315080024A801FA03F2D8F8343823EA0203C8F83438AC
S315080024B808EB4613C3F8081923698B42ADD0594669
S315080024C8204602F0A3FB2369012BAFD1002EADD11C
S315080024D8C6EBC602930023441B6D002BA6D104F550
S315080024E871720121206801F031FC9FE731462046C8
S315080024F8FFF790FCBDE7D5F8043823F00103C5F8C3
S31508002508043894F8F433012B08D0204602F0C4FBAB
S315080025182268536903F000435361A2E6002184F850
S31508002528F413204600F09EFAF2E7204602F09AFBDA
S31508002538A3E6204602F096FBC0E605F50069D9F839
S31508002548043023F00103C9F804301021206800F08C
S31508002558BDFF14E008EB47134FF67F31C3F8081997
S31508002568D3F8002922F40012C3F80029C3F8081B77
S31508002578D3F8002B22F40012C3F8002B013763683E
S315080025889F42E7D3D9F81C3043F00113C9F81C3029
S31508002598236BEBB1D9F8843043F00B03C9F88430C0
S315080025A8D9F8443043F00B03C9F84430D5F8003855
S315080025B823F4FE63C5F8003804F57172217C206897
S315080025C801F0C4FB2268536903F4805353617CE61F
S315080025D8D9F8142042F22B031343C9F81430D9F852
S315080025E8103043F00B03C9F81030DFE7206801F014
S315080025F891FB206801F072F8E060276800F034FA69
S31508002608227B0146384600F0C7FE204602F010FB3A
S315080026182268536903F4005353615DE647F6F0737D
S315080026281F423FF46FAE4FEAC80AAAEB08034FEAFF
S315080026388309A1443F09C7F30A02D9F808122846AC
S3150800264801F078FAC7F30A07D9F808323B44C9F8FB
S315080026580832D9F814321F44C9F8147252E6082207
S3150800266804F57171284601F065FAC7F30A174FEAA7
S31508002678C803A3EB08018A002244D2F814321F447F
S31508002688C2F814723EE6204602F0CBFA226853696D
S3150800269803F00803536141E6F1B2204602F00BFB4A
S315080026A82268536903F4801353613EE6F1B2204663
S315080026B802F0FBFA2268536903F4001353613BE6F8
S315080026C8204602F0FEFA2268536903F080435361F4
S315080026D839E6204602F0FFFA42E690F8BC33012BA9
S315080026E801D10220704710B50446012380F8BC338F
S315080026F8006801F0C2FA002084F8BC0310BD90F8FF
S31508002708BC33012B01D10220704710B504460123BA
S3150800271880F8BC33006801F0BCFA002084F8BC03D2
S3150800272810BD90F8BC33012B01D10220704710B5B3
S315080027380446012380F8BC3380F83810006801F095
S315080027488CFA002084F8BC0310BDF8B511F0800F88
S315080027581ED101F00F06F500AF1BBC00274604F58D
S31508002768FC74044404343E460644002586F8FD51A4
S3150800277801F00F012170A260E370627802B1E1806E
S31508002788022B14D090F8BC33012B13D10220F8BDC4
S3150800279801F00F06F500AF1BBC0027463834044481
S315080027A804343E460644012586F83D50E0E70023F2
S315080027B82371E7E70546012380F8BC3321460068FC
S315080027C800F09CFF002085F8BC03F8BD38B511F069
S315080027D8800F17D101F00F04E200151BAB001D4648
S315080027E803F5FC73034404332C460444002284F896
S315080027F8FD2101F00F01197090F8BC23012A10D1A8
S31508002808022038BD01F00F04E200151BAB001D4677
S315080028183833034404332C460444012284F83D2003
S31508002828E7E70446012280F8BC231946006800F049
S31508002838ADFF002084F8BC0338BD70B501F00F055C
S31508002848EE00711B8C0004F5FC740444211D761BEC
S31508002858B4000444C4F80822C4F810320023C4F8A3
S31508002868143284F8FD3184F8FC510369012B06D02B
S3150800287865B1DAB2006801F069F8002070BDC5EBE9
S31508002888C506B4000444C4F80C22F1E7DAB20068B5
S3150800289800F0C4FFF1E701F00F01C1EBC1018B009D
S315080028A81844D0F81402704770B501F00F05EE0009
S315080028B8711B8C0038340444211D761BB40004446B
S315080028C8A264236500236365012384F83D3084F8F0
S315080028D83C500369012B06D05DB1DAB2006801F0F5
S315080028E835F8002070BDC5EBC506B4000444E2649B
S315080028F8F2E7DAB2006800F091FFF2E738B501F0BE
S315080029080F0543689D4238D811F0800F15D1CA00C3
S31508002918541AA3001C4603F5FC73034404332246E1
S315080029280244002182F8FD1101229A701D7090F860
S31508002938BC23012A0DD1022038BDEA00511B8B00A1
S3150800294819463833034404330144012281F83D20EB
S31508002958EAE70446012280F8BC231946006801F014
S31508002968FDF81DB1002084F8BC0338BD04F5717262
S31508002978217C206801F0EAF9F4E7012038BD01F066
S315080029880F03426893422FD810B511F0800F14D15F
S31508002998DA00D41AA1000C4601F5FC710144043189
S315080029A80444002284F8FD2100228A700B7090F8EE
S315080029B8BC33012B0DD1022010BDDA00D41AA100B0
S315080029C80C463831014404310444012284F83D2078
S315080029D8EAE70446012380F8BC33006801F0EBF8FF
S315080029E8002084F8BC0310BD0120704730B4046881
S315080029F8606A29B10D46A36A00EB134000230CE070
S31508002A0840EA0240A06212E003F1400104EB8101AA
S31508002A18496800EB11400133DBB2691E8B42F3D3D8
S31508002A2840EA024005F13F0104EB810148600020B5
S31508002A3830BC70470368596200207047024603682D
S31508002A480121C0F8FC13002082F8F4039A6942F0C1
S31508002A5800629A61596D024A0A435A65704700BF6F
S31508002A680300001070470000014B1868704700BF44
S31508002A7808000020534B98421FD0534B984228D041
S31508002A88524B984231D0524B98423AD0514B9842C1
S31508002A9843D0514B98424CD0504B984255D0504B46
S31508002AA898425ED04F4B984267D04F4B984270D0A9
S31508002AB84E4B984279D00120704703F560531A693E
S31508002AC842F001021A611A6922F001021A6100200D
S31508002AD8704703F550531A6942F002021A611A69D7
S31508002AE822F002021A610020704703F540531A695A
S31508002AF842F004021A611A6922F004021A610020D7
S31508002B08704703F530531A6942F008021A611A69C0
S31508002B1822F008021A610020704703F520531A6943
S31508002B2842F010021A611A6922F010021A6100208E
S31508002B38704703F510531A6942F020021A611A6998
S31508002B4822F020021A610020704703F500531A691B
S31508002B5842F040021A611A6922F040021A610020FE
S31508002B68704703F5E0531A6942F080021A611A6938
S31508002B7822F080021A610020704703F5C0531A69CB
S31508002B8842F480721A611A6922F480721A61002066
S31508002B98704703F5A0531A6942F400721A611A6954
S31508002BA822F400721A610020704703F580531A69E7
S31508002BB842F480621A611A6922F480621A61002056
S31508002BC8704700BF000002400004024000080240A7
S31508002BD8000C02400010024000140240001802408F
S31508002BE8001C02400020024000240240002802403F
S31508002BF8F0B40C6894FAA4F4B4FA84F42BE08E685A
S31508002C08826893FAA3F5B5FA85F56D0007FA05F50E
S31508002C1822EA050293FAA3F5B5FA85F56D0006FAD0
S31508002C2805F52A43826037E04A69456A1B0A93FA1A
S31508002C38A3F6B6FA86F6B6000F2707FA06F625EAC1
S31508002C48060593FAA3F3B3FA83F39B0002FA03F390
S31508002C582B43436201340B6833FA04F250D001223D
S31508002C68A2401340F6D04E68026893FAA3F5B5FA5F
S31508002C7885F56D00032707FA05F522EA050293FA92
S31508002C88A3F5B5FA85F56D0006FA05F52A43026037
S31508002C984A68013A012AB2D90E69C26893FAA3F5B5
S31508002CA8B5FA85F56D00032707FA05F522EA050240
S31508002CB893FAA3F5B5FA85F56D0006FA05F52A43DC
S31508002CC8C2604A68022AC5D193FAA3F2B2FA82F216
S31508002CD8072AA9D84D69026A93FAA3F6B6FA86F6B8
S31508002CE8B6000F2707FA06F622EA060293FAA3F3AE
S31508002CF8B3FA83F39B0005FA03F313430362A9E7C0
S31508002D084A68013A012A02D90020F0BC7047C96806
S31508002D18426822EA030201FB03F313434360F3E71D
S31508002D281E4A136843F0010313601C4B1B6813F013
S31508002D38020FFAD0194A00239360194B13601368D7
S31508002D4823F0F80343F080031360144B1B6813F051
S31508002D58007FFAD1114B1B6813F0006FFAD10F4B9D
S31508002D681B6813F0005FFAD10C4B0E4A5A60103AEA
S31508002D78C3F88420C3F88820DA6822F4FE42DA60A9
S31508002D88DA6842F47F02DA605A6F22F001025A675B
S31508002D985A6F42F080725A6700207047003802401E
S31508002DA8FFFFF2EA10300024034B9B68C3F30313B2
S31508002DB8024AD35CD840704700380240D850000809
S31508002DC8034B9B68C3F38223024AD35CD8407047F7
S31508002DD800380240E8500008034B9B68C3F34233A7
S31508002DE8024AD35CD840704700380240E8500008C9
S31508002DF80D4B5B6803F480030BB90C4800E00C48DC
S31508002E08094A536803F03F03B0FBF3F35068C0F36D
S31508002E18881000FB03F05368C3F3014301335B00D2
S31508002E28B0FBF3F0704700BF003802400024F400F6
S31508002E3800127A0008B5074B9B6803F00C03042BAD
S31508002E4806D0082B01D0044808BDFFF7D1FF08BDF6
S31508002E58024808BD003802400024F40000127A002F
S31508002E6810B50446FFF7E6FF2060FFF79DFF606090
S31508002E78FFF7A6FFA0606068FFF7AEFFE06010BD29
S31508002E8808B5032809D00C2833D0B0F5406F5CD0B4
S31508002E98302800F08780002008BD584BD3F89030BA
S31508002EA8034043EA0040564B98420FD0B0F1031F3F
S31508002EB815D0013B984206D0FFF7BCFFFFF774FF11
S31508002EC8FFF78AFF08BDFFF7B5FF08BD4B4B1B6820
S31508002ED813F0020F01D04B4808BD002008BD474B28
S31508002EE81B6F13F0020F02D04FF4004008BD0020F4
S31508002EF808BD424BD3F89030034043EA0040424BA2
S31508002F0898420FD0B0F10C1F15D0043B984206D052
S31508002F18FFF790FFFFF748FFFFF752FF08BDFFF7D7
S31508002F2889FF08BD354B1B6813F0020F01D03548D9
S31508002F3808BD002008BD314B1B6F13F0020F02D0E5
S31508002F484FF4004008BD002008BD2C4BD3F890303C
S31508002F58034043EA00402D4B984210D0B0F10C2F9D
S31508002F6816D0A3F58063984206D0FFF763FFFFF7EC
S31508002F781BFFFFF731FF08BDFFF75CFF08BD1F4BB6
S31508002F881B6813F0020F01D01E4808BD002008BDB3
S31508002F981A4B1B6F13F0020F02D04FF4004008BDFE
S31508002FA8002008BD154BD3F89030034043EA00408B
S31508002FB8174B98420FD0B0F1301F15D0103B9842E6
S31508002FC806D0FFF737FFFFF7EFFEFFF7F9FE08BD54
S31508002FD8FFF730FF08BD094B1B6813F0020F01D035
S31508002FE8084808BD002008BD044B1B6F13F0020FE4
S31508002FF802D04FF4004008BD002008BD0038024042
S31508003008020003000024F40008000C000008000C65
S315080030182000300008B5C0280BD0B0F5407F34D062
S31508003028B0F5405F5ED0B0F5404F00F088800020CC
S3150800303808BD594BD3F89030034043EA0040574B34
S3150800304898420FD0B0F1C01F15D0403B984206D021
S31508003058FFF7F0FEFFF7A8FEFFF7B2FE08BDFFF779
S31508003068E9FE08BD4C4B1B6813F0020F01D04C480B
S3150800307808BD002008BD484B1B6F13F0020F02D08D
S315080030884FF4004008BD002008BD434BD3F89030E4
S31508003098034043EA0040434B984210D0B0F1032F4F
S315080030A816D0A3F58073984206D0FFF7C3FEFFF73C
S315080030B87BFEFFF785FE08BDFFF7BCFE08BD364B4D
S315080030C81B6813F0020F01D0354808BD002008BD5B
S315080030D8314B1B6F13F0020F02D04FF4004008BDA6
S315080030E8002008BD2C4BD3F89030034043EA004033
S315080030F82D4B984210D0B0F1302F16D0A3F5805337
S31508003108984206D0FFF796FEFFF74EFEFFF758FEE1
S3150800311808BDFFF78FFE08BD1F4B1B6813F0020F8B
S3150800312801D01F4808BD002008BD1B4B1B6F13F0B4
S31508003138020F02D04FF4004008BD002008BD164B08
S31508003148D3F89030034043EA0040184B984210D011
S31508003158B0F1C02F16D0A3F58043984206D0FFF7E2
S3150800316869FEFFF721FEFFF72BFE08BDFFF762FE93
S3150800317808BD094B1B6813F0020F01D0084808BDA3
S31508003188002008BD044B1B6F13F0020F02D04FF442
S31508003198004008BD002008BD003802408000C00075
S315080031A80024F4000002000300200030008000C05C
S315080031B838B5036813F0010F46D00123002B77D1E1
S315080031C80D46044603683D4A1A404B68C9680B43CE
S315080031D829690B43A9690B4313430360AB68426823
S315080031E822F44052134343606B69826822F44072A2
S315080031F813438360324B984228D0324B984229D0E1
S31508003208314B98422AD0314B98422BD0304B9842B2
S315080032182CD0304B98422ED02F4B984230D02F4B7B
S31508003228984232D00020002844D02B68002B43D07F
S31508003238AA69B2F5004F2DD000EB5300B0FBF3F0A6
S3150800324880B2E060002038BD0023B7E70320FFF707
S3150800325817FEE8E70C20FFF713FEE4E73020FFF730
S315080032680FFEE0E7C020FFF7D5FEDCE74FF4407015
S31508003278FFF7D0FED7E74FF44060FFF701FED2E725
S315080032884FF44050FFF7C6FECDE74FF44040FFF72E
S31508003298C1FEC8E75A0802EB4000B0FBF3F04FF648
S315080032A8F0730340C0F342001843E060002038BDBD
S315080032B8012038BD012038BD012038BDF369FFEF6C
S315080032C8001001400044004000480040004C0040FF
S315080032D8005000400014014000780040007C00407F
S315080032E8002301330C4A934211D80269002AF8DAF6
S315080032F8036943F00103036100230133064A934235
S3150800330807D8026912F0010FF7D100207047032089
S3150800331870470320704700BF400D030084B010B5FE
S31508003328044603A880E80E00089B012B11D0E36821
S3150800333843F04003E3602046FFF7D2FFA36B43F44C
S315080033488033A363069B012B1BD0BDE8104004B04D
S315080033587047A36B23F48033A363E2680D4B1340CD
S31508003368E360E36823F44013E3600F9B012B03D063
S315080033782046FFF7B5FFE5E7E36843F48013E36003
S31508003388F6E7A36843F00603A360A36843F020039F
S31508003398A360DAE7BFFFBDFF022A0AD00921C2687F
S315080033A822F47052C260C36843EA8123C3600020CE
S315080033B87047274B0B44274A934239D9264B0B4467
S315080033C8264A934236D9264B0B44264A934233D982
S315080033D8254B0B4402F5C332A03293422ED9234B10
S315080033E80B44234A93422BD9224B0B4402F59222CB
S315080033F802F57872934225D91F4B0B4402F5C3226E
S3150800340802F5207293421FD91C4B0B4402F5B712DA
S3150800341802F55872934219D9194B0B4402F5122230
S3150800342802F5F862934201D90621B8E70721B6E7FB
S315080034380F21B4E70E21B2E70D21B0E70C21AEE75C
S315080034480B21ACE70A21AAE70921A8E70821A6E77C
S31508003458405327FFFF340C00401E1BFF3F420F0056
S3150800346800DC0BFF7F4F1200808CF9FE60B6E5FE84
S315080034785FE3160000D3CEFEC05BB3FE00CA91FE1A
S31508003488E05459FE836843F00103836000207047BF
S31508003498836823F0010383600020704708B5C36872
S315080034A823F0C043C360012909D069B9C36843F04A
S315080034B88043C3603220FEF707F8002008BDC368BA
S315080034C843F00053C360F5E7012008BD890141F0C0
S315080034D82001016100230133054A934205D8026990
S315080034E812F0200FF7D1002070470320704700BF5D
S315080034F8400D03001023036100230133054A934254
S3150800350805D8026912F0100FF7D10020704703207A
S31508003518704700BF400D0300D0F800381943C0F8BB
S31508003528001800207047000084B02DE9F0410446D1
S3150800353807A880E80E002546002306E003F14002A6
S3150800354804EB82020021516001330E2BF6D9119B38
S3150800355883BBA36B23F40013A363236843F04003D8
S315080035682360236843F0800323600023C4F8003EE1
S3150800357804F50066D4F80038C4F800380C9B012B0B
S315080035881DD0032B27D003212046FFF7C5FF10219E
S315080035982046FFF79BFF804608B14FF001082046F2
S315080035A8FFF7A8FF08B14FF00108002333617361DC
S315080035B8F36127E0A36B43F40013A363D5E7099BDC
S315080035C823B900212046FFF7A7FFE0E70121204697
S315080035D8FFF7A2FFDBE7099B23B900212046FFF77F
S315080035E89BFFD4E701212046FFF796FFCFE7C3B92B
S315080035F84FF00060C2F8000900220A614FF67F32D0
S315080036088A60013307998B4210D205EB431202F5FB
S315080036181061D2F800090028E9DB0020C2F8000981
S31508003628EAE74FF09040C2F80009E5E700230AE008
S31508003638BBB14FF09047C2F8007B002202614FF6F3
S315080036487F32826001338B4210D205EB431202F5B2
S315080036583060D2F8007B002FEADB0027C2F8007B2F
S31508003668EBE74FF00067C2F8007BE6E7336923F417
S31508003678807333610A9B012B1BD00022A2616FF06D
S31508003688804262611BB9A36943F01003A361A2696A
S315080036980E4B1343A3610D9B1BB1A36943F00803A3
S315080036A8A361119B012B0BD04046BDE8F04104B03D
S315080036B87047074A3263316B064A0A433263DCE7C6
S315080036C8A269054B1343A361EEE700BF00383C80A7
S315080036D8000180000300010004000040D0F8083803
S315080036E813F0060305D0062B18BF022B03D10220B8
S315080036F870470020704700207047000070B40B78A8
S315080037084A78012A20D0D0F81C2803F00F0601248D
S31508003718B44042EA0442C0F81C2800EB4310D0F82B
S31508003728003B13F4004F0CD1D0F8002B8B68C3F379
S315080037380A03C97843EA81431343134A1A43C0F86C
S31508003748002B002070BC7047D0F81C4803F00F0601
S31508003758B24092B22243C0F81C2800EB4310D0F8B6
S31508003768002912F4004FECD1D0F800498A68C2F350
S315080037780A02C97842EA814242EA83532343024A43
S315080037881A43C0F80029DCE70080001070B40C78EA
S315080037984B78012B1FD0D0F83C5804F00F060122AD
S315080037A802FA06F625EA0645C0F83C58D0F81C5829
S315080037B8097801F00F018A4025EA0242C0F81C2858
S315080037C800EB4410D0F8002B124B1340C0F8003B0E
S315080037D8002070BC7047D0F83C6804F00F0203FA62
S315080037E802F292B226EA0202C0F83C28D0F81C284F
S315080037F8097801F00F018B409BB222EA0303C0F84F
S315080038081C3800EB4410D0F80029034B1340C0F8C5
S315080038180039DDE70078F3EF007833EC70B40B78FD
S315080038284C78012C24D000EB431000F530631D6951
S315080038383A4C2C401C611D69394C2C401C614C695A
S315080038480CB18C684C611C6944F400241C611C6921
S315080038588D68C5F312052C431C61012A59D0D0F886
S31508003868003B43F00443C0F8003B002070BC704797
S315080038784C6954BB00EB4314D4F81069284D3540FD
S31508003888C4F81059D4F8105945F40025C4F8105945
S31508003898D4F81069214D3540C4F81059012A30D09A
S315080038A84A694AB1D0F83428097801F00F04012189
S315080038B8A1400A43C0F8342800EB4310D0F8002981
S315080038C842F00442C0F80029CFE700EB431404F598
S315080038D810642669114D354025612669104D354015
S315080038E825614E698D68AE4200D94D61256945F452
S315080038F80025256125694E69C6F3120635432561F3
S31508003908CCE70A69002AD7D000EB4311C1F8142975
S31508003918D2E7CA68002AA2D05A61A0E70000F8FFD1
S31508003928FFFF07E070B49DF80C4064B903339E089E
S3150800393807E000EB023303F5805351F8045B1D607A
S315080039480134B442F5D3002070BC7047F0B583B093
S315080039580C784B78012B29D000EB441404F5306316
S315080039681E69714D35401D611E69704D35401D61D2
S315080039784D69002D40F0AA801D698E68C6F31206A7
S3150800398835431D611D6945F400251D61012A00F0AE
S31508003998B280CB78012B00F0B480D4F8003B43F012
S315080039A80443C4F8003B002003B0F0BD4B69002B64
S315080039B83BD100EB4413D3F810695C4D3540C3F886
S315080039C81059D3F8105945F40025C3F81059D3F8F7
S315080039D81069554D3540C3F81059012A57D0CB7888
S315080039E8012B0BD04B694BB1D0F834380D7805F05C
S315080039F80F060125B5402B43C0F83438CB78012B80
S31508003A084DD000EB4414D4F8003943F00443C4F805
S31508003A180039CB78012BC6D114460B46C9681A78E3
S31508003A289B8A0094FFF77EFFBDE700EB4413D3F8A3
S31508003A3810693D4D3540C3F81059D3F810693B4D08
S31508003A483540C3F81059D3F810694D698F683D4455
S31508003A58013DB5FBF7F5364F07EAC5453543C3F8C3
S31508003A681059D3F810594E69C6F312063543C3F8E8
S31508003A78105903F51063CD78012DAED11D6925F0CF
S31508003A88C0451D611D6945F000551D61A5E70B690F
S31508003A98002BB3D000EB4415C5F81439AEE7D0F8B7
S31508003AA8083813F4807F08D100EB4415D5F8003997
S31508003AB843F00053C5F80039A3E700EB4415D5F8D9
S31508003AC8003943F08053C5F800399AE78E683544BB
S31508003AD8013DB5FBF6F51E69154F07EAC5473E438E
S31508003AE81E611F698E68ADB206FB05F5C5F312059A
S31508003AF83D431D614AE7CA68002A3FF44AAF5A613E
S31508003B0847E7D0F8083813F4807F06D1D4F8003B85
S31508003B1843F00053C4F8003B3FE7D4F8003B43F0B2
S31508003B288053C4F8003B38E70000F8FFFFFF07E0BA
S31508003B380000F81F03329208002393420CD210B4EF
S31508003B4800F58054246841F8044B01339342F7D3AF
S31508003B5808465DF8044B7047084670470B784A785C
S31508003B68012A14D000EB4310D0F8002B002A06DBF4
S31508003B782BB1D0F8003B23F08043C0F8003BD0F8BF
S31508003B88003B43F40013C0F8003B0020704700EBE5
S31508003B984310D0F80029002A06DB2BB1D0F80039E3
S31508003BA823F08043C0F80039D0F8003943F40013ED
S31508003BB8C0F80039E9E70B784A78012A0ED000EBF5
S31508003BC84310D0F8003B23F40013C0F8003BCB7829
S31508003BD8023BDBB2012B15D90020704700EB4310D6
S31508003BE8D0F8003923F40013C0F80039CB78023B23
S31508003BF8DBB2012BF0D8D0F8003943F08053C0F86F
S31508003C080039E9E7D0F8003B43F08053C0F8003B99
S31508003C18E2E738B505460446002208E004EB4213F5
S31508003C284FF67F31C3F80819C3F8081B01320E2A64
S31508003C38F4D90022C5F81028C5F81428C5F81C2890
S31508003C482846FFF757FC034608B1184638BD102121
S31508003C582846FFF73BFC0346F7E7D0F8003823F475
S31508003C68FE63C0F80038D0F80038090101F4FE618F
S31508003C780B43C0F800380020704708B5D0F8043858
S31508003C8823F00203C0F804380320FDF71DFC0020C2
S31508003C9808BD08B5D0F8043843F00203C0F804385C
S31508003CA80320FDF711FC002008BD42698069104011
S31508003CB87047D0F8183800F50060C0691840000C3D
S31508003CC87047D0F8183800F50060C069184080B207
S31508003CD8704700EB4111D1F8082B00F500604069E0
S31508003CE81040704710B4D0F81028D0F8343801F0CE
S31508003CF80F04E340DB01DBB2134300EB4111D1F8B3
S31508003D08080918405DF8044B7047406900F001003F
S31508003D1870470000D0F800290B4B1340C0F800394B
S31508003D2800F500639A6802F00602042A05D05A6864
S31508003D3842F480725A6000207047D0F8002942F091
S31508003D480302C0F80029F2E700F8FFFF10B4046C74
S31508003D58154B9C4203D9D0F8003B002B16DB0024F0
S31508003D68C0F8104BD0F8104B44F40024C0F8104B98
S31508003D78D0F8104B44F01804C0F8104BD0F8104B84
S31508003D8844F0C044C0F8104B012903D000205DF860
S31508003D98044B7047C0F8142BD0F8003B43F0802337
S31508003DA8C0F8003BF2E700BF0A30544F014B1860D1
S31508003DB8704700BF0800002098B108B50346D0F838
S31508003DC88C0210B10020C3F88C0209B1C3F8881216
S31508003DD81846012380F87432027000F087FF002025
S31508003DE808BD0220704710B50446012380F87432CE
S31508003DF8D0F88C325B6801799847204600F0E6FFD0
S31508003E08204600F0D3FF002010BD19B1C0F88C1267
S31508003E18002070470220704708B500F0CFFF002041
S31508003E2808BD08B5D0F88C3223B11B68984718B175
S31508003E38022008BD022008BD002008BD08B5D0F834
S31508003E488C325B689847002008BD38B5044600F5EB
S31508003E582075284600F049F90123C4F86C32B4F8ED
S31508003E688632C4F8703294F8801201F01F03012BC9
S31508003E780ED03BB1022B10D001F08001204600F08D
S31508003E88C0FF03E02946204600F0B9FA002038BDED
S31508003E982946204600F0E7FAF8E72946204600F0C2
S31508003EA812FBF3E738B50446A9BB1046D4F86C32BA
S31508003EB8032B03D0052B25D0002038BDD4F84C3168
S31508003EC8D4F8502193420DD99B1AC4F84C319A421A
S31508003ED806D99AB20146204600F030FC002038BDC3
S31508003EE892B2F7E7D4F88C321B691BB194F874229E
S31508003EF8032A04D0204600F029FC002038BD2046B5
S31508003F089847F7E70025C4F86C522946204600F07A
S31508003F1878FF284638BD0A46D0F88C329B694BB1DB
S31508003F2890F87412032901D0022038BD1146984723
S31508003F38002038BD022038BD10B50446002956D1E0
S31508003F481046D4F86C32022B09D0002B18BF042B64
S31508003F5844D094F87832012B45D0002010BD236A46
S31508003F68626A93421BD8E169B1FBF2F302FB1313A9
S31508003F782BB98A4203D8D4F8703299421DD3D4F89B
S31508003F888C32DB681BB194F87422032A23D080216B
S31508003F98204600F036FF204600F0E3FBD9E79A1AD8
S31508003FA8226292B20146204600F0C0FB00231A4658
S31508003FB81946204600F045FFCBE700221146204661
S31508003FC800F0B4FB0021C4F870120B460A462046D6
S31508003FD800F037FFBDE720469847D8E780212046F6
S31508003FE800F00FFFB5E7002084F8780210BD0A46EE
S31508003FF8D0F88C325B694BB190F87412032901D05A
S31508004008022010BD11469847002010BD022010BD99
S3150800401870B5044640230022114600F0DFFE01254C
S31508004028C4F844514026C4F850613346002280211A
S31508004038204600F0D3FEA561666284F87452002310
S31508004048C4F86C326360C4F87C32D4F890322BB169
S31508004058D4F88C325B68002120469847002070BD4A
S3150800406801740020704790F8743280F8753204237A
S3150800407880F874320020704790F8753280F87432E8
S315080040880020704708B590F87432032B01D0002039
S3150800409808BDD0F88C32DB69002BF8D09847F6E7CC
S315080040A800207047002070470020704708B5012295
S315080040B880F87422D0F88C2252680179904700203B
S315080040C808BD002302E00133DBB201300278002A7A
S315080040D8F9D11846704708B54B88012B00D008BD9A
S315080040E8C0F87C3200F032FBF9E70B7803704B789E
S315080040F843708B78CA7803EB022343800B794A7995
S3150800410803EB022383808B79CA7903EB0223C380E6
S31508004118704710B50446802100F073FE002120463A
S3150800412800F06FFE10BD30B583B005460C464A88C8
S31508004138130A013B062B00F28480DFE803F0041615
S315080041482A8282667300D0F888321B680DF1060148
S31508004158007C9847BDF8062012B1E388002B74D175
S31508004168E388002B7BD003B030BD037C43B9D0F875
S315080041788C329B6A0DF10600984702234370E9E7DB
S31508004188D0F88C32DB6A0DF1060098470223437093
S31508004198E0E7D2B2052A34D8DFE802F0030B131B8E
S315080041A8232BD0F888325B680DF10601007C984706
S315080041B8D0E7D0F888329B680DF10601007C98474D
S315080041C8C8E7D0F88832DB680DF10601007C984705
S315080041D8C0E7D0F888321B690DF10601007C9847BC
S315080041E8B8E7D0F888325B690DF10601007C984774
S315080041F8B0E7D0F888329B690DF10601007C98472C
S31508004208A8E72146FFF785FFADE7037C33B9D0F861
S315080042188C325B6B0DF1060098479BE72146FFF742
S3150800422878FFA0E7037C43B9D0F88C321B6B0DF1F5
S3150800423806009847072343708CE72146FFF769FF6E
S3150800424891E72146FFF765FF8DE79A4228BF1A4688
S31508004258ADF806200146284600F05BFA80E72846AE
S3150800426800F074FA7FE738B504468B88F3B9CB882B
S31508004278E3B94B887F2B19D803F07F0590F8743279
S31508004288032B0CD080F87652294600F0CAFD204642
S3150800429800F05CFA35B1022384F8743238BDFFF7AA
S315080042A838FF38BD012384F8743238BD2046FFF735
S315080042B830FF38BD38B504460D468978284B19703D
S315080042C801290ED890F87432022B0ED0032B21D070
S315080042D82946FFF71EFF224B19782046FFF7AEFD41
S315080042E838BD2946FFF715FF38BD81B1416003235C
S315080042F880F87432FFF795FD022803D0204600F0AF
S3150800430825FA38BD29462046FFF703FF38BD00F0D1
S315080043181DFA38BD89B1436899421DD0D9B2FFF74D
S315080043288DFD0F4B197861602046FFF77AFD022844
S315080043380DD0204600F00AFA38BD022380F87432F8
S315080043484160FFF77BFD204600F000FA38BD294694
S315080043582046FFF7DEFE38BD00F0F8F938BD00BF85
S31508004368D409002008B5CB88012B0BD190F87432F4
S315080043789BB1022B09D9032B0FD10122011D00F08D
S31508004388C8F908BDFFF7C5FE08BD0146002341F870
S31508004398083F012200F0BDF908BDFFF7BAFE08BDBF
S315080043A808B590F87432013B022B12D8CB88022B39
S315080043B80CD10123C360D0F87C320BB10323C36048
S315080043C8022200F10C0100F0A4F908BDFFF7A1FECE
S315080043D808BDFFF79EFE08BD08B590F87432013B84
S315080043E8022B09D84B88012B00D008BD0023C0F83A
S315080043F87C3200F0ABF908BDFFF78BFEF5E708B588
S315080044080B7803F06003202B05D0402B03D043B16B
S31508004418FFF77FFE03E0D0F88C329B6898470020A8
S3150800442808BD4B78092B1BD8DFE803F011171A14B7
S315080044381A08051A0E0BFFF776FEF0E7FFF713FFC3
S31508004448EDE7FFF737FFEAE7FFF78CFFE7E7FFF740
S31508004458A7FFE4E7FFF73FFEE1E7FFF7BDFFDEE763
S31508004468FFF757FEDBE738B505460C460B7803F029
S315080044786003202B05D0402B03D013B1FFF749FE64
S315080044880BE095F87432013B022B17D82379012BD8
S3150800449805D921462846FFF73CFE002038BDD5F841
S315080044A88C329B68214628469847E388002BF4D126
S315080044B80028F2D1284600F049F9EEE721462846B1
S315080044C8FFF727FEE9E738B504468A880B7803F02C
S315080044D86003202B08D0D0B2402B05D05BB120460C
S315080044E8FFF717FE002038BDD4F88C329B682046A3
S315080044F89847002038BD202B12D04B78012B3AD08C
S31508004508002B67D0032B40F0E18094F87432022B15
S315080045180CD0032B1DD02046FFF7FBFD002038BD25
S31508004528D4F88C329B682046984738BD002818BFAF
S31508004538802809D00146204600F063FC80212046E1
S3150800454800F05FFC002038BD2046FFF7E2FD00209A
S3150800455838BD4B882BB9002818BF802801D0CB88CE
S3150800456823B1204600F0F2F8002038BD014620465F
S3150800457800F047FCF5E794F87432022B06D0032BB3
S3150800458817D02046FFF7C5FD002038BD002818BFFC
S31508004598802809D00146204600F033FC80212046B1
S315080045A800F02FFC002038BD2046FFF7B2FD00209A
S315080045B838BD4B88002B40F08E8010F07F0F04D151
S315080045C8204600F0C3F8002038BD0146204600F012
S315080045D820FCF5E794F87432022B06D0032B2AD070
S315080045E82046FFF796FD002038BD002818BF80280A
S315080045F812D112F0800F14D100F07F0000EB800072
S31508004608830003F5A073E11800250D6002222046F1
S3150800461800F07FF8284638BD2046FFF77AFD0020C7
S3150800462838BD00F07F0000EB8000830003F110011D
S3150800463821440431E8E752B2002A1FDB00F00F03D1
S3150800464803EB83039D002544D5F8443123B3002A98
S3150800465827DB00F07F0202EB8202930003F5A073C2
S31508004668E518802818BF002825D100232B600222C8
S315080046782946204600F04DF8002038BD00F00F0303
S3150800468803EB83039D002544AB69002BDFD1204645
S31508004698FFF73FFD002038BD2046FFF73AFD00200A
S315080046A838BD00F07F0202EB8202930003F1100581
S315080046B825440435D5E70146204600F051FB10B1DC
S315080046C801232B60D3E700232B60D0E72046FFF7AA
S315080046D820FD002038BD002038BDC8B170B50D468C
S315080046E816460446FFF7EDFC013040003080287076
S315080046F803236B70022307E05A1CD2B20134E9542B
S315080047080233DBB20021A95421780029F4D170BDFF
S31508004718704710B513460222C0F86C22C3610362BB
S315080047280A46002100F085FB002010BD08B513468F
S315080047380A46002100F07DFB002008BD08B513468F
S315080047480A46002100F07DFB002008BD08B50423B1
S31508004758C0F86C3200231A46194600F06AFB002096
S3150800476808BD08B50523C0F86C3200231A46194651
S3150800477800F067FB002008BD10B40F4AD2F888304D
S3150800478843F47003C2F888300C4B196841F00101EC
S315080047981960002098601C68094921401960094970
S315080047A85960196821F480211960D8604FF00063B0
S315080047B893605DF8044B704700ED00E0003802404E
S315080047C8FFFFF6FE1030002408B52F4A136823F0B9
S315080047D80F0343F007031360136803F00F03072B4F
S315080047E803D06A212948FCF7CDFA294B1A6842F4FE
S315080047F840421A601A6842F480321A6003F5E433B4
S315080048081A6842F480221A601A6842F480321A60DA
S31508004818204B1B6813F4003FFAD01E4B5A681E49F2
S3150800482811401E4A0A435A605A681D4911401D4AD2
S315080048380A435A601A6842F080721A60154B1B6858
S3150800484813F0007FFAD0134B9A6822F0F0029A60A8
S315080048589A6822F4E05242F4A0529A609A6822F4BE
S31508004868604242F400429A609A6822F0030242F0D3
S3150800487802029A60074B9B6803F00C03082BF9D1D0
S315080048880948FFF793FA08BD003C0240F0500008B3
S3150800489800700040003802400080BCFF086C4000E9
S315080048A80080BFF0086C400900E6DF0C08B5FCF785
S315080048B8FFFDFFF789FF08BD08B5FFF7F7FFFCF707
S315080048C8AFFAFCF7BBFAFCE72DE9F04391B04C4C7C
S315080048D8636C43F480436364636C03F4804309930D
S315080048E8099B236C43F080532364236C03F080539D
S315080048F80893089B236B43F001032363236B03F098
S3150800490801030793079B236B43F002032363236B77
S3150800491803F002030693069B236B43F00403236301
S31508004928236B03F004030593059B236B43F00803E5
S315080049382363236B03F008030493049B236C43F453
S3150800494880232364236C03F480230393039B236C3B
S3150800495843F000732364236C03F000730293029BED
S3150800496880230A9301230B9300250C950D950E9524
S31508004978DFF89C800AA94046FEF73AF94FF4000387
S31508004988C8F818304FF400530A930B950E950AA9E0
S315080049981C48FEF72DF94FF44079CDF828900227E0
S315080049A80B9703260C960D950E9507230F930AA9C0
S315080049B81548FEF71DF9CDF828900B970C960D9516
S315080049C80E9509230F930AA94046FEF711F94FF4E5
S315080049D8C0530A930B970C960D950E950A230F93B9
S315080049E80AA90A48FEF704F9636B43F08003636370
S315080049F8636B03F080030193019B11B0BDE8F08354
S31508004A080038024000080240000C0240000002403C
S31508004A180004024010B5FEF783F91B4C4FF4000357
S31508004A28A3611A48FEF726F81948FEF723F8204620
S31508004A38FEF720F81748FEF71DF8174B5A6B22F0B1
S31508004A4880025A631A6C22F000721A641A6C22F4ED
S31508004A5880221A641A6B22F008021A631A6B22F06B
S31508004A6804021A631A6B22F002021A631A6B22F0FE
S31508004A7801021A631A6C22F080521A645A6C22F4DC
S31508004A8880425A6410BD00BF00040240000C024070
S31508004A98000802400000024000380240DFF834D01F
S31508004AA8002103E00C4B5B58435004310B480C4B70
S31508004AB842189A42F6D30B4A02E0002342F8043B0E
S31508004AC8094B9A42F9D3FFF757FE00F053FAFFF756
S31508004AD8F3FE704700000520585100080000002022
S31508004AE8C0000020C00000203C100020FEE700009F
S31508004AF82023038000487047440000200A230380C7
S31508004B08004870476400002008B590F87432032BF3
S31508004B1801D0002008BDFCF7D5F8FAE708B5FCF778
S31508004B28D1F8002008BD08B50846FCF7FFF80020AC
S31508004B3808BD000008B50B7813F0600F06D14B784E
S31508004B480A2B14D00B2B17D0062B01D0002008BD32
S31508004B584B881B0A212B04D00B491722FFF7D9FDCE
S31508004B68F4E7CA88172A28BF17220849F6E7012250
S31508004B780749FFF7CEFDE9E78B7813B9044A1360AE
S31508004B88E4E7FFF7C6FAE1E74D00002056000020E3
S31508004B98D809002010B50446812100F02AF9012118
S31508004BA8204600F026F9002010BD000010B504467E
S31508004BB840230222812100F011F940230222012113
S31508004BC8204600F00BF94023034A0121204600F04D
S31508004BD838F9002010BD00BFF809002000487047C2
S31508004BE8F809002008B500F57171D0F80004FFF738
S31508004BF82CF908BD08B5C1EBC10293000344D3F8E4
S31508004C080822D0F80004FFF74DF908BD08B5C1EB2E
S31508004C18C102930003449A6CD0F80004FFF78CF994
S31508004C2808BD08B5D0F80004FFF72CFA08BD00003F
S31508004C3810B50446C3683BB1022B0FD0912108482A
S31508004C48FCF7A0F8012100E00021D4F80004FFF7DA
S31508004C5807FAD4F80004FFF7DBF910BD0121F4E7D9
S31508004C68FC50000810B50446D0F80004FFF7FBF915
S31508004C782268D2F8003E43F00103C2F8003E236AD0
S31508004C8823B1044A136943F006031361FCF79CFB36
S31508004C9810BD00BF00ED00E010B50446FCF795FB13
S31508004CA8D4F80004FFF7E8F910BD08B5D0F80004F1
S31508004CB8FFF7F8F908BD08B5D0F80004FFF7F0F9CA
S31508004CC808BD10B504460120FCF77DFBD4F800049E
S31508004CD8FFF7EAF910BD10B504460020FCF773FB88
S31508004CE8D4F80004FFF7E2F910BD000003780BB109
S31508004CF80020704710B503461748C0F80034C3F8B3
S31508004D0898024FF0A0430360062343600222C2605C
S31508004D180023036182610122C26103624362C3629E
S31508004D280363FDF7E1F880B90B4C80212046FDF7AF
S31508004D3881FE402200212046FDF758FE80220121E7
S31508004D482046FDF753FE002010BD40F22511034802
S31508004D58FCF718F8E8E700BF380A0020FC500008F6
S31508004D68D0F8983211F0800F08D101F07F01C1EB15
S31508004D78C1018A00134493F8FE01704701F07F01C8
S31508004D88C1EBC1018A00134493F83E00704708B581
S31508004D98D0F89802FDF77FFD08BD18B1022803D0A0
S31508004DA802207047002070470120704708B5D0F8E0
S31508004DB89802FDF760F9FFF7F0FF08BD08B5D0F8C7
S31508004DC89802FDF723F9FFF7E8FF08BD08B5D0F8FC
S31508004DD89802FDF730F9FFF7E0FF08BD10B51C4645
S31508004DE813462246D0F89802FDF7AFFCFFF7D5FF21
S31508004DF810BD08B5D0F89802FDF7E8FCFFF7CDFF17
S31508004E0808BD08B5D0F89802FDF778FDFFF7C5FF85
S31508004E1808BD08B5D0F89802FDF7B1FDFFF7BDFF44
S31508004E2808BD08B5D0F89802FDF77BFCFFF7B5FF73
S31508004E3808BD08B5D0F89802FDF736FDFFF7ADFFAF
S31508004E4808BD08B5D0F89802FDF7F7FCFFF7A5FFE7
S31508004E5808BD000012230B80004870478C0000200C
S31508004E6804230B8000487047A000002000239342C3
S31508004E7816D230B40BE0373401F8134000015C0051
S31508004E88013400250D550133DBB2934206D2040FCF
S31508004E98092CF0D8303401F81340EFE730BC7047D6
S31508004EA87047000038B50A4B186804331C68043381
S31508004EB81B68C01800D138BD064D0822A91CFFF783
S31508004EC8D5FF042205F112012046FFF7CFFFF2E7C6
S31508004ED820F4F01FA400002008B51A230B80FFF75A
S31508004EE8E1FF014808BD00BFA400002008B50A462E
S31508004EF828B105490548FFF7F0FB034808BD0249EC
S31508004F080248FFF7EAFBF8E73C0E00203C51000888
S31508004F1810B5044C0A4621460348FFF7DEFB20462F
S31508004F2810BD00BF3C0E00202C51000808B50A46E3
S31508004F3828B105490548FFF7D0FB034808BD0249CB
S31508004F480248FFF7CAFBF8E73C0E00200C51000898
S31508004F5808B50A4628B105490548FFF7BEFB0348C0
S31508004F6808BD02490248FFF7B8FBF8E73C0E0020DF
S31508004F781451000870B50D4E0D4CA41BA41000253D
S31508004F88A54209D10B4E0C4C00F018F8A41BA41026
S31508004F980025A54205D170BD56F825309847013534
S31508004FA8EEE756F8253098470135F2E750510008DC
S31508004FB8505100085051000854510008F8B500BF70
S31508004FC8F8BC08BC9E467047F8B500BFF8BC08BCD4
S30908004FD89E4670472C
S31508004FDC2E2E5C2E2E5C2E2E5C2E2E5C536F75722E
S31508004FEC63655C41524D434D375F53544D333246DE
S31508004FFC375C63616E2E630005020602060307031F
S3150800500C0803090309040A040B040C040C050D0512
S3150800501C0E050F050F06100610071008008000086D
S3150800502C008000000100000000000108008000005C
S3150800503C0200000000800108008000000300000048
S3150800504C000002080000020004000000000004082A
S3150800505C0000040005000000000008080000040019
S3150800506C0600000000000C08000004000700000001
S3150800507C2E2E5C2E2E5C2E2E5C2E2E5C536F75728D
S3150800508C63655C41524D434D375F53544D3332463D
S3150800509C375C72733233322E630000002E2E5C2E70
S315080050AC2E5C2E2E5C2E2E5C536F757263655C41DE
S315080050BC524D434D375F53544D333246375C7573F7
S315080050CC622E63004F70656E424C5400000000005F
S315080050DC000000000102030406070809000000008E
S315080050EC010203042E2E5C6D61696E2E63000000AE
S315080050FC2E2E5C757362645F636F6E662E6300009A
S3150800510C44656661756C740057696E555342204246
S3150800511C756C6B20496E7465726661636500000078
S3150800512C4F70656E424C5420557365720000000032
S3150800513C57696E5553422042756C6B2044657669E7
S3090800514C6365000089
S30908005150ED01000857
S30908005154C901000877
S3150800515804010000100000000024F400B54B000804
S315080051689D4B00083D4B00080000000000000000A9
S31508005178254B00082F4B0008114B000800000000BB
S315080051880000000000000000F94A000800000000BE
S31508005198054B000809022000010100C03209040075
S315080051A80002FF000000070581024000FF0705010D
S315080051B8024000FF0A060002000000400100000045
S315080051C85D4E0008694E0008194F0008F54E00089C
S315080051D8E14E0008354F0008594F00081201000231
S315080051E800000040501DAC600002010203010000E7
S315080051F8040309041A030000000000000000000068
S315080052080000000000000000000000000000000088
S70508004AA503
